:100000000C9400280C9402280C9404280C940628C4
:100010000C9408280C940A280C940C280C940E2894
:100020000C9410280C9412280C9414280C94162864
:100030000C9418280C941A280C941C280C941E2834
:100040000C9420280C9422280C9424280C94262804
:100050000C9428280C942A280C942C280C942E28D4
:100060000C943028FFFFFFFFFFFFFFFFFFFFFFFFA4
:10007000FFFFFFFFFFFFFFFFFFFFFFFFFFFFFFFF90
:10008000FFFFFFFFFFFFFFFFFFFFFFFFFFFFFFFF80
:10009000FFFFFFFFFFFFFFFFFFFFFFFFFFFFFFFF70
:1000A000FFFFFFFFFFFFFFFFFFFFFFFFFFFFFFFF60
:1050000033C0000046C0000044C0000042C00000A1
:1050100040C000003EC000003CC000003AC000009C
:1050200038C0000036C0000034C0000032C00000AC
:1050300030C000002EC000002CC000002AC00000BC
:1050400028C0000026C0000024C0000022C00000CC
:1050500020C000001EC000001CC000001AC00000DC
:1050600018C0000016C0000011241FBECFEFD8E00A
:10507000DEBFCDBF11E0A0E0B1E0E0E0F4E602C0A9
:1050800005900D92A230B107D9F70E9422310C94FD
:10509000FE31B6CFBF92CF92DF921F93CF93DF93B3
:1050A000DC01CB01142FE901E4E3F8E30F921F9236
:1050B0007EEF6AE956E540E8D92EC82EBA2E212F98
:1050C0001D2E0C2E09952131F9F71F900F90DF91BD
:1050D000CF911F91DF90CF90BF900895BF92CF9254
:1050E000DF921F93CF93DF93DC01CB01142FE901F3
:1050F000E4E3FFE30F921F927EEF6AE956E540E892
:10510000D92EC82EBA2E212F1D2E0C2E09952131F5
:10511000F9F71F900F90DF91CF911F91DF90CF9003
:10512000BF900895CF93DF93FA01E901213831054B
:1051300010F0C0E8D0E0AB01BC0140789E01CF0187
:105140000E941931CE01DF91CF9108952F923F92A5
:105150004F925F926F927F928F929F92AF92BF9287
:10516000CF92DF92EF92FF920F931F93CF93DF9333
:1051700000D01F92CDB7DEB7D42E2A833B832A817D
:105180003B812138310520F0E0E8F0E0FB83EA8341
:105190002A803B803694279430E8432E55245A9435
:1051A000652C752C462257226822792220E030E0B7
:1051B00043E0C301B2015983F8010995ED2C5981EF
:1051C000F52E53014201C12CD12C11C0F7012191C0
:1051D00031917F0141E0C501B401F8010995F2E088
:1051E0008F0E911CA11CB11C2FEFC21AD20AC2143F
:1051F000D30461F720E030E045E0C301B201F801DB
:1052000009958A819B810F900F900F90DF91CF912C
:105210001F910F91FF90EF90DF90CF90BF90AF90D4
:105220009F908F907F906F905F904F903F902F90C6
:10523000089542C4000075C4000059C4000057C45A
:10524000000055C4000053C4000051C400004FC406
:1052500000004DC400004BC4000049C4000047C416
:10526000000045C4000043C4000041C400003FC426
:1052700000003DC400003BC4000039C4000037C436
:10528000000035C4000033C4000031C400002FC446
:1052900000002DC400002BC400007E3FF9F76A39DE
:1052A000F9F75635F9F74038F9F7EC2DFD2DB7B67B
:1052B000B0FCFDCF27BFE895B7B6B0FCFDCF21E12C
:1052C000B7B6B6FCF4CF08955553426173704C6F76
:1052D000616465722076302E39362E322062792054
:1052E0005374657068616E2042616572776F6C6699
:1052F00020286D617472697873746F726D40676D88
:10530000782E6465292C2053636877616E73656518
:1053100020323031330A687474703A2F2F6D617403
:1053200072697873746F726D2E636F6D2F61767210
:105330002F74696E79757362626F6172642FFFFFFB
:10534000FFFFFFFFFFFFFFFFFFFFFFFFFFFFFFFF6D
:10535000FFFFFFFFFFFFFFFFFFFFFFFFFFFFFFFF5D
:10536000FFFFFFFFFFFFFFFFFFFFFFFFFFFFFFFF4D
:10537000FFFFFFFFFFFFFFFFFFFFFFFFFFFFFFFF3D
:105A6000FFFFFFFFFFFF0902120001010080320962
:105A7000040000000000000012011001FF000008F7
:105A8000C016DC050201010200010E03550053009F
:105A900042006100730070001C03770077007700FC
:105AA0002E00660069007300630068006C002E0021
:105AB000640065000403090411241FBECFEFD8E081
:105AC000DEBFCDBF11E0A0E0B1E0E8EFFFE702C02C
:105AD00005900D92A830B107D9F721E0A8E0B1E018
:105AE00001C01D92AE33B207E1F771D19CC3A1CBC7
:105AF000A82FB92F80E090E041E050EA609530E0B7
:105B000009C02D9182279795879510F084279527B6
:105B1000305EC8F36F5FA8F30895EADF8D939D931D
:105B20000895CF93CFB7CF93DF93C3954F9BE9F7FA
:105B30004F9B0BC04F9B09C04F9B07C04F9B05C09D
:105B40004F9B03C04F9B01C089C06F93C09121013F
:105B5000DD27C85DDE4F2F9365E54F9B03C02F9176
:105B60006F91E6CF0F931F934F9320E040E15F9337
:105B700009B1047807FB27F93F9350E03BE039C0B7
:105B8000147840642F77012F5F5F1EC0406819B101
:105B900014782F7752501FC0406409B12F770478D2
:105BA000D1F15F5F00C023C0406219B12F77147834
:105BB00091F15F5F00C025C004781027515012F4A6
:105BC0005D5F0000115027952C3F19B1C8F614787D
:105BD0000127015027952C3FC8F64227499309B168
:105BE000047810274F73115027952C3FA8F646953F
:105BF000469519B1147879F00127015027952C3F6B
:105C000098F66B5A60F3315009B1B0F600C011E05C
:105C10001CBB002717C03B503195C31BD04011E07F
:105C20001CBB0881033CF9F00B34E9F020911F0103
:105C30001981110F1213EDCF093651F10D3211F008
:105C4000013E39F7009326013F915F914F911F91DB
:105C50000F912F916F91CCB3C0FD67CFDF91CF91A2
:105C6000CFBFCF91189520912601222369F310917F
:105C70002401112339F534303AF130932401209373
:105C80002001109121013BE0311B309321011CC008
:105C9000009124010130B4F40AE53091010134FD92
:105CA00014C000930101C4E1D1E013C0052710E046
:105CB00000C000000BB91AC0052710E0221F1DC04C
:105CC00010E021C04AE502C032ED432FC4E1D0E02C
:105CD00032E01AB114685F9A0BB11AB954E820E89F
:105CE00065E320FF05270BB9279517951C3FF0F6B4
:105CF0006695B8F7B1F720FF05270BB927951795DB
:105D00001C3FD0F62795179517FF052700001C3F6D
:105D10000BB9B0F629913A9519F70B771091250137
:105D2000110FC651D0400BB911F010931F0111E0B3
:105D30001CBB00681AB11B77402F4B7754E05A9573
:105D4000F1F70BB91AB94BB97FCFFC013381932F0F
:105D50004481842F2281203339F44370E42FF0E012
:105D6000ED5FFE4F80810895283529F431110EC072
:105D7000E1E0F0E006C0203599F431110CC0E0E01C
:105D8000F0E089E080935700849108953830E9F479
:105D9000E3E0F0E0F6CF3830C1F4E2E0F0E0F1CF3C
:105DA000203221F4FC01EE0FFF1F06C0283231F42F
:105DB000FC01EE0FFF1F319684910895203A09F4FB
:105DC0001CC2203C11F4658120D280E008951AB8ED
:105DD00080E48BB914BE81E085BF82E085BF8FE38C
:105DE0009CE90197F1F700C000004E9B0EC0F894AB
:105DF000579A1BB81DBA1092690081E085BF15BE85
:105E0000E0911201F0911301099584B7877F84BF57
:105E100088E10FB6F89480936000109260000FBE86
:105E200080916900826080936900E89A579A9FEF99
:105E3000E1EBFCE09150E040F040E1F700C00000F1
:105E40005798789400912401035007FD3BC180913D
:105E50002101CCE0D0E0C81BD109C85DDE4F8091A4
:105E600020018D3209F0B7C0083009F029C183EC58
:105E7000809314018AE580930101109208018881C2
:105E8000807629818823B9F189E091E090932301FC
:105E900080932201233031F4CE0157DF80930C012F
:105EA00024E08FC0253019F12A3009F1822F845067
:105EB000863098F48A819B8190930E0180930D0126
:105EC0002930B9F08E8180930F018D81827080938B
:105ED0001001209311012FEF6DC08091000122303D
:105EE00011F48E7F01C081608093000102C021E027
:105EF00068C020E066C08A8110921D01211106C091
:105F000010921E018DE191E022E04EC0253019F47F
:105F1000809325013DC02630A9F59B81913019F46D
:105F200086E498E704C0923041F484E398E79093C4
:105F300023018093220122E121C09330F1F48111E9
:105F400008C082E898E7909323018093220124E01F
:105F500015C0813041F486E698E790932301809341
:105F600022012CE10BC0823041F488E598E7909340
:105F70002301809322012EE001C020E080E4809381
:105F8000080116C0283069F0293029F480932701D0
:105F90008DE191E004C08DE191E02A3021F020E014
:105FA00003C087E291E021E09093230180932201D6
:105FB0002F3F39F4888187FD2E8180E88093080186
:105FC00007C08F81811104C08E81821708F4282FA9
:105FD0002093020175C08091080187FF71C08091F4
:105FE0000F01801708F4082F801B80930F01FF24F6
:105FF000F3948111F12C10E05DC02091110180918A
:106000000D0190910E01273058F069919C012F5F8E
:106010003F4F30930E0120930D01F7D01F5F4AC010
:106020008115904708F04AC01E5FF894E0910D0179
:10603000F0910E018991999121E00C012093570074
:10604000E8951124789480910D0190910E010296AB
:1060500090930E0180930D018F779927892B41F042
:10606000FF2041F1101730F180911001882311F1C8
:10607000F894E0910D01F0910E01329783E0809346
:106080005700E895789407B600FCFDCFF894E091AE
:106090000D01F0910E01329785E080935700E8954D
:1060A000789407B600FCFDCFF89481E18093570007
:1060B000E8957894101708F4A0CFF110109202011F
:1060C000109224018091010184FF73C0809102012C
:1060D0008F3F09F46EC0F82E893010F028E0F22EC0
:1060E0008F19809302018091140198E88927809389
:1060F0001401FF2009F44BC08091080187FF28C0DC
:1061000080910F018F1508F4F82E8F1980930F01DD
:10611000E0901101C5E1D1E014C000910D01109192
:106120000E0186E08E1518F4C80167D002C0F80190
:106130008491888321960F5F1F4F10930E01009367
:106140000D0185E191E0FC2FF81BFF1530F31CC019
:10615000E0912201F0912301A5E1B1E086FF09C0A1
:1061600084918D93319685E191E08F0D8A13F8CF5C
:1061700007C081918D9385E191E08F0D8A13F9CF4E
:10618000F0932301E093220128E02F1560F06F2D9A
:1061900085E191E0C2DC8F2D8C5F8C3041F09FEF68
:1061A0009093020104C08FEF809302018EE18093EF
:1061B000010184E199B1947831F48150D9F71092BA
:1061C000250110921F0180910001803130F04E9B1B
:1061D0000FC080910001805109C04E9909C0809183
:1061E0000001823028F080910001825080930001EC
:1061F00080910001811126CEFACDF999FECF92BD92
:1062000081BDF89A992780B50895262FF999FECF78
:106210001FBA92BD81BD20BD0FB6F894FA9AF99AC3
:106220000FBE01960895F894FFCFFE5AFF1E950FFA
:106230000000FA01DC0102C005900D9221503040AF
:10624000D8F70895AF92BF92CF92DF92EF92FF926C
:106250000F931F93CF93DF93CDB7DEB7C058D1090B
:106260000FB6F894DEBF0FBECDBF88E10FB6F8942D
:1062700080936000109260000FBEF89488E28AB9A3
:1062800083E084B980E28BB91982209100013091BA
:10629000010180E090E0F901E80FF91F6591749128
:1062A000FC01F059459154916417750719F081E08C
:1062B000898305C00296811540E1940761F78981C1
:1062C000882309F488C068E6C62E60E7D62EE12C44
:1062D000F12C20E830E0AE014F5F5F4FC701B601FF
:1062E0000E9492289C01C701B6016856724F8F4FD9
:1062F0009F4F0AE418E2AE014F5F5F4F0E94A6284D
:1063000080E8C80ED11CE11CF11C48E6C41642E727
:10631000D406E104F104E9F6C12C50E7D52EE12CB6
:10632000F12C560180E7B81A40910001509101010B
:106330004A0D5B1D662757FD6095762F20E830E0FB
:10634000CE01019676DF0EE618E220E830E0AE01DD
:106350004F5F5F4FC701B6010E94A62840E8C40EF8
:10636000D11CE11CF11CC11483E7D806E104F1043F
:10637000C1F6E12C40E1F42EEA18FB08970141E850
:10638000E416F10410F020E830E040910001509153
:1063900001014A0D5B1D662757FD6095762FCE01E2
:1063A000019647DFB501705980E090E00AE418E2F9
:1063B00020E830E0AE014F5F5F4F0E94A62880E8E2
:1063C000A80EB11C40E8E41AF108A11480E1B80657
:1063D000A8F282E085B9289AC058DF4F0FB6F8942A
:1063E000DEBF0FBECDBFDF91CF911F910F91FF9008
:1063F000EF90DF90CF90BF90AF900895F894FFCFCB
:10640000325218E20E94B42880E890E0A80EB91E2B
:10641000A0E8BFEFCA0EDB1EB0E0AB16B0E1BB06D2
:1064200088F282E085B9289AC058DF4F0FB6F894F9
:10643000DEBF0FBECDBFDF91CF911F910F91FF90B7
:10644000EF90DF90CF90BF90AF900895F894FFCF7A
:106450005C52FFFFFFFFFFFFFFFFFFFFFFFFFFFF9C
:10646000FFFFFFFFFFFFFFFFFFFFFFFFFFFFFFFF3C
:10647000FFFFFFFFFFFFFFFFFFFFFFFFFFFFFFFF2C
:10648000FFFFFFFFFFFFFFFFFFFFFFFFFFFFFFFF1C
:10649000FFFFFFFFFFFFFFFFFFFFFFFFFFFFFFFF0C
:00000001FF
